:020000040800F2
:100000000006022001020008190F00081D0F000859
:10001000750F00081D0F0008490F000803020008B3
:10002000030200080302000803020008692900080F
:10003000030200080302000803020008030200088C
:10004000030200080302000803020008030200087C
:100050000302000803020008553A0008813A00082C
:10006000AD3A0008D93A0008053B00080302000831
:10007000030200080302000803020008030200084C
:10008000030200080302000803020008030200083C
:10009000030200080302000803020008313B0008C5
:1000A000030200080302000803020008030200081C
:1000B0007938000803020008030200080302000860
:1000C00003020008030200080302000803020008FC
:1000D0000302000803020008291100083D1100086E
:1000E000993B00080302000803020008030200080D
:1000F00003020008030200080302000803020008CC
:1001000003020008030200080302000803020008BB
:1001100003020008030200080302000803020008AB
:10012000030200080302000803020008030200089B
:10013000030200080302000803020008030200088B
:10014000030200080302000803020008D53000087B
:10015000030200080302000803020008030200086B
:10016000030200080302000803020008030200085B
:10017000030200080302000803020008030200084B
:1001800003020008030200085111000803020008DE
:10019000030200080302000803020008030200082B
:1001A000030200080302000803020008030200081B
:1001B000030200080302000803020008030200080B
:1001C00003020008030200080302000803020008FB
:1001D00003020008030200080302000803020008EB
:1001E00003020008030200080302000803020008DB
:1001F00003020008030200080302000803020008CB
:1002000002E000F000F8FEE772B6394880F3088893
:10021000384880F3098838484EF60851CEF200017C
:10022000086040F20000CCF200004EF63471CEF2CD
:1002300000010860BFF34F8FBFF36F8F40F20000E3
:10024000C0F2F0004EF68851CEF200010860BFF314
:100250004F8FBFF36F8F4FF00000E1EE100A4EF6A4
:100260003C71CEF200010860062080F31488BFF3D1
:100270006F8F02F0B7FB03F087FA4FF055301F493C
:100280001B4A91423CBF41F8040BFAE71C49194A4A
:1002900091423CBF41F8040BFAE71A491A4A1B4B3A
:1002A0009A423EBF51F8040B42F8040BF8E70020D5
:1002B0001749184A91423CBF41F8040BFAE702F093
:1002C000D5FB03F0CBFA144C144DAC4203DA54F8CE
:1002D000041B8847F9E700F03FF8114C114DAC4280
:1002E00003DA54F8041B8847F9E702F0BDBB0000AD
:1002F0000006022000220220000000080000022068
:100300000006022010400008002202205022022095
:1003100050220220343502200002000800020008AA
:1003200000020008000200082DE9F04F2DED108AB0
:10033000C1F80CD0D0F80CD0BDEC108ABDE8F08F1D
:10034000002383F311882846A047002001F094FF82
:1003500001F0B2FE00DFFEE770B578231F4C0025E8
:100360006FF07F0623701E236570A570E570257100
:100370006571A571E57125726672A372E57200F070
:10038000DFFC20B10E2325726672A372E57202F0C3
:10039000ADFA044602F0E2FA0546D0B9104B9C4291
:1003A00019D001339C4241F2883412BF0546002423
:1003B0000125002002F0A4FA0DB100F05BF800F076
:1003C0004DFD00F001FC204600F0F4F800F052F87A
:1003D000F9E70024EDE70446EBE700BF50220220D6
:1003E000010007B008B500F06DFBA0F120035842F2
:1003F000584108BD054B07B51B88022101A8ADF87F
:10040000043000F0CBFB03B05DF804FB803C000837
:1004100010B5202383F311881248C3680BB101F093
:10042000B1FF0023104A4FF47A710E4801F06EFFBD
:10043000002383F311880D4C236813B12368013B1B
:100440002360636813B16368013B6360084B1B78EA
:1004500033B9636823B9022000F078FC322363606B
:1004600010BD00BF5C220220110400087823022086
:1004700070220220454B46492DE9F04153F8042FE4
:10048000013201D1BDE8F0818B42F7D1414C424BA2
:1004900022689A4278D9414B9B6803F1006303F5C7
:1004A000C0339A4270D2002000F0AAFB02203C4BDD
:1004B000187000F049FC3B4B1A6C00221A64196E4C
:1004C0001A66196E596C5A64596E5A66596E596992
:1004D00041F080015961596921F0800159615969E0
:1004E000196941F000511961196921F00051196130
:1004F0001B6972B62C4B2D490B601D682468BFF335
:100500004F8FBFF36F8F2A4BC3F88420BFF34F8FF9
:100510005A6922F480325A61BFF34F8FD3F880209A
:1005200043F6E07EC2F3C906C2F34E32B70752016A
:1005300002EA0E0838463146013948EA000C00F15B
:100540004040B1F1FF3FC3F874C2F5D1203A12F137
:10055000200FEDD1BFF34F8FBFF36F8FBFF34F8FDE
:10056000BFF36F8F5A6922F400325A610022C3F838
:100570005022BFF34F8FBFF36F8F202383F3118877
:10058000AD4685F308882047BDE8F081FC7F01086F
:100590001C80010804800108FF7F0108502202200E
:1005A00070220220003802400080010808ED00E0BF
:1005B00000ED00E02DE9F04F99B0B34C2022FF216F
:1005C000019010A8A66800F0EBFBB04AA346137890
:1005D000A3B90121AE481170C360202383F31188B1
:1005E000C3680BB101F0CEFE0023AA4A4FF47A7122
:1005F000A74801F08BFE002383F31188019B13B100
:10060000A54B019A1A600023A44AA349019F994669
:100610001C461D46984613704B600292012000F064
:1006200093FB002F00F012829B4B1B68002B40F0C5
:100630000D8219B0BDE8F08F0220FFF7D3FE00282D
:1006400040F0FB81019BB9F1000F08BF1F46944B9E
:100650001B8802210BA8ADF82C3000F09FFADDE7D3
:100660004FF47A7000F02EFA031E0393EADB0220A7
:10067000FFF7B8FE82460028E4D0039B581E0428EA
:1006800000F2DD81DFE800F0030E1114170018A856
:100690000523042140F8343D00F080FA54464FF021
:1006A000000856E004217848F6E704217D48F3E786
:1006B00004217D48F0E71C242046043400F0A2FA0F
:1006C00004210B900BA800F069FA2C2CF4D1E5E77B
:1006D000002DB7D0002CB5D00220FFF783FE0546D1
:1006E000002800F0AF8101206C4C00F089FA4FF037
:1006F00000090220207000F027FB5FFA89FA5046BB
:1007000000F08EFA074658B1504609F1010900F091
:1007100097FA0028F1D12C46A9460027634B97E7AA
:1007200001233E460220237000F00CFBDBF808306A
:100730009E4206D2304600F065FA0130EBD1043615
:10074000F4E70026029BA9462C461E703746524B02
:100750005E6000F079FB15B1002C18BF0027FFF791
:1007600049FE5BE7002D3FF46DAF002C3FF46AAF0C
:100770000220029B187000F0E7FA322000F0A2F984
:10078000B0F1000AC0F25E811AF0030540F05A8110
:1007900006EB0A03DBF80820934200F25381BAF516
:1007A000807F00F24F8155450DDA4FF47A7000F0EA
:1007B00089F90490049B002BC0F24481049B3C4ABD
:1007C000AB540135EFE7C820FFF70CFE05460028C3
:1007D00000F038811F2E11D8C6F1200410AB26F08E
:1007E000030033495445184428BF5446224600F0BC
:1007F000AFFA2246FF212E4800F0D2FA4FEAAA0AA9
:100800002B4930465FFA8AF200F0D2FA04460028FB
:1008100000F01A8106EB8A0605469AE70220FFF7E8
:10082000E1FD00283FF40EAF00F030FA00283FF45D
:1008300009AF4FF0000A5346DBF8082092451CD25E
:10084000BAF11F0F12D8109A01320FD02AF003020A
:1008500018A90A4452F8202C0B92184604220BA91E
:100860000AF1040A00F09AFB0346E5E750460393B9
:1008700000F0C8F9039B0B90EFE718A8042140F89B
:100880004C3D00F08BF964E75022022074230220D3
:100890005C2202201104000878230220702202202A
:1008A000823C00085422022058220220843C000886
:1008B0007422022018A80023642140F8343D00F07F
:1008C00039F900287FF4BEAE0220FFF78BFD002827
:1008D0003FF4B8AE0B9800F0C5F918AB43F8480DDB
:1008E00004211846CDE718A80023642140F8343DC0
:1008F00000F020F900287FF4A5AE0220FFF772FD7A
:1009000000283FF49FAE0B9800F0BAF918AB43F8FB
:10091000440DE5E70220FFF765FD00283FF492AEA5
:1009200000F0C4F918AB43F8400DD9E70220FFF7F7
:1009300059FD00283FF486AE0BA9142000F0BCF945
:10094000824618A8042140F83CAD00F027F9514632
:100950000BA896E7322000F0B5F8B0F1000AFFF6D8
:1009600071AE1AF0030F7FF46DAE0AEB0803DBF8EB
:10097000082093423FF666AE0220FFF733FD0028C1
:100980003FF460AE2AF0030AC244D0453FF4E1AE22
:10099000404608F1040800F035F904210A900AA83D
:1009A00000F0FCF8F1E74FF47A70FFF71BFD002828
:1009B0003FF448AE00F06AF900283FF4AFAE109B58
:1009C00001330CD0082210A9002000F0F1F9002812
:1009D0003FF4A4AE2022FF2110A800F0E1F9FFF7B8
:1009E00009FD374801F04EFC23E6002D3FF42AAE06
:1009F000002C3FF427AE18A80023642140F8343DB2
:100A000000F098F8824600287FF41CAE0220FFF721
:100A1000E9FC00283FF416AE0390FFF7EBFC41F22F
:100A20008830574601F02EFC0B9800F055FA00F084
:100A30000BFA039B1C461D46F0E5054689E64FF080
:100A40000008FFE52546FDE52C4667E6002000F09E
:100A500039F80490049B002BFFF6E3AD012000F071
:100A600071F9049B213B122B3FF6D8AD01A252F83D
:100A700023F000BF3906000861060008D10600080F
:100A80001D0600081D0600081D0600086507000871
:100A9000550900081D080008B5080008E708000807
:100AA000150900081D0600082D0900081D0600088C
:100AB000A7090008530700081D060008EB090008F5
:100AC000A08601002DE9F3474FF47A75002402AEA9
:100AD000154F4543DFF8588006F8014D97F900306F
:100AE0005FFA84F95A1C01D0A34212D158F82400AD
:100AF000012231460368D3F820A02B46D0470128B5
:100B000007D10A4B9DF8070083F8009002B0BDE8BA
:100B1000F0870134042CE1D14FF4FA7001F0B2FBFC
:100B20004FF0FF30F2E700BF00220220C423022072
:100B3000883C00082DE9F0474FF47A7506460024FA
:100B4000134F4D43DFF8508097F900305FFA84F976
:100B50005A1C01D0A34210D158F824000422314677
:100B60000368D3F820A02B46D047042805D1094BB1
:100B7000002083F80090BDE8F0870134042CE3D115
:100B80004FF4FA7001F07EFB4FF0FF30BDE8F087C4
:100B900000220220C4230220883C0008074B30B406
:100BA0001A78074B53F822400A460146236820462C
:100BB000DD69044BAC4630BC604700BFC423022053
:100BC000883C0008A0860100F8B50A4C00250A4EB2
:100BD00001F092FD094F207030682378834207D9D5
:100BE00001F084FD336805440133BD423360F3D91D
:100BF000F8BD00BFC523022080230220FF7F010033
:100C000001F026BE00F1006000F5C03000687047BA
:100C100000F10060920000F5C03001F0B3BD0000AB
:100C2000054B1A68054B1B789B1A834202D9104466
:100C300001F05CBD0020704780230220C523022004
:100C400038B5074D04462868204401F057FD28B9FF
:100C500028682044BDE8384001F068BD38BD00BFB9
:100C60008023022010F0030308D1B0F5806F05D86F
:100C700000F10050A0F57120006870470020704717
:100C8000014BC058704700BF20F4F01F064991F88F
:100C9000243033B100230822086A81F82430FFF79A
:100CA000B7BF0120704700BF84230220014B1868A2
:100CB000704700BF002004E01F4BF0B51E681F4BBB
:100CC000C6F30B02360C1F885D68BA4293F90840E0
:100CD00022D09F89BA4221D01F8BBA4206D102226C
:100CE0000C2404FB02335D6893F90840B6F5805F7D
:100CF00016D041F201039E4208BF5A24421E013D14
:100D00000B460A44934215D215F9016F581C4EB197
:100D1000034600F8016CF5E70022E1E70122DFE776
:100D20004124EBE72C2582421D7001D9981C5C7090
:100D3000401AF0BD1846FBE7002004E00422022020
:100D400000207047704700007047000070470000A7
:100D5000002310B5934203D0CC5CC4540133F9E7AF
:100D600010BD000030B5441E14F9010F0B4658B1F8
:100D700093F900500131854206D11AB993F9002048
:100D8000801A30BD013AEFE7002AF7D1104630BD96
:100D900002460346981A13F9011B0029FAD170473D
:100DA00002440346934202D003F8011BFAE770475E
:100DB0002DE9F047234C05468846174694F8243021
:100DC00083BB2E46DFF87C90C7B394F824302BB950
:100DD0002022FF2148462662FFF7E2FF94F8240014
:100DE0004146C0F1080504EB8000BD4228BF3D46E6
:100DF0005FFA85FAAD00A7EB0A072A462E44FFF7F3
:100E0000A7FF94F82430A844FFB29A445FFA8AFA04
:100E1000BAF1080F84F824A0D6D1FFF737FF0028D5
:100E2000D2D108E0266A06EB8306B042CAD0FFF7AB
:100E30002DFF0028C5D10020BDE8F0870120BDE8C6
:100E4000F08700BF84230220024B1A78024B1A70ED
:100E5000704700BFC423022000220220F8B5184CBE
:100E6000184800F0BDFC2146164800F0E5FC246857
:100E70001548E26E154DD2F80438154E43F00203C2
:100E8000104FC2F8043801F0FDF92046114900F076
:100E9000E1FDE26E0024D2F8043823F00203C2F828
:100EA00004384FF4E1332B6056F82400B84202D0E6
:100EB000294600F0F3FB0134042CF5D1F8BD00BF46
:100EC000A83D0008482D022040420F00AC2302201C
:100ED000883C0008D43D000838B50B4B05461A780D
:100EE0000A4B53F822400A4B9C420CD0094B00217C
:100EF00018221846FFF754FF056001462046BDE85A
:100F0000384000F0CBBB38BDC4230220883C000829
:100F1000482D0220AC230220FEE7000000B59BB064
:100F2000EFF3098168226846FFF712FFEFF30583AC
:100F3000044B9A6BDA6A9A6A9A6A9A6A9A6A9A6A05
:100F40009B6AFEE700ED00E000B59BB0EFF309817E
:100F500068226846FFF7FCFEEFF30583044B9A6BAB
:100F60009A6A9A6A9A6A9A6A9A6A9B6AFEE700BFC4
:100F700000ED00E000B59BB0EFF309816822684600
:100F8000FFF7E6FEEFF30583034B5A6B9A6A9A6A02
:100F90009A6A9A6A9B6AFEE700ED00E030B50A445F
:100FA000074D91420BD011F8013B09245840013CF8
:100FB000F7D040F300032B4083EA5000F7E730BD41
:100FC0002083B8ED002304491A465A50C818083344
:100FD0004260802BF9D17047C82302200268436821
:100FE0001143016003B1184770470000024A1368BB
:100FF00043F0C0031360704700440040024A136886
:1010000043F0C0031360704700480040024A136871
:1010100043F0C00313607047007800402DE9F047AB
:10102000C66D05463768F469200734621AD014F09B
:10103000080F0CBF00218021E20748BF41F02001CA
:10104000A3074FF0200348BF41F04001600748BFAD
:1010500041F4807183F31188281DFFF7BFFF00233F
:1010600083F31188E2050AD5202383F311884FF416
:101070000071281DFFF7B2FF002383F311884FF0A2
:1010800020094FF0000A14F0200831D13B0616D594
:101090004FF0200905F1380A200610D589F3118890
:1010A000504600F06FFA00282FDA0821281DFFF7BC
:1010B00095FF27F080033360002383F311887906BE
:1010C0000DD562060BD5202383F31188EA6C2B6DB6
:1010D0009A4201D12B6CEBB9002383F31188E3060C
:1010E00020D5AA6E1369EBB15069BDE8F0471847E7
:1010F00089F31188736A284695F86410194000F046
:10110000DBFA8AF31188F469BDE7B06288F31188CD
:10111000F469C1E727F040071021281DFFF75EFFA3
:101120003760D9E7BDE8F08708B50348FFF776FFD9
:10113000BDE8084001F028BC4824022008B5034857
:10114000FFF76CFFBDE8084001F01EBCB42402208C
:1011500008B50348FFF762FFBDE8084001F014BC82
:101160002025022037B52D4C2D4D204600F08AFA5F
:10117000009404F1140000234FF48072294900F018
:101180004BF94FF48072009404F13800264B274944
:1011900000F0C4F9264B25660B21E3652620254C7B
:1011A00000F0C4F8204600F06DFA009404F1140039
:1011B00000234FF48072204900F02EF94FF4807222
:1011C000009404F138001D4B1D4900F0A7F91D4B98
:1011D00025660B21E36527201B4C00F0A7F820466D
:1011E00000F050FA04F11400009400234FF48072D0
:1011F000164900F011F904F1380000944FF48072A0
:10120000134B144900F08AF9134B0B215220E3656C
:10121000256603B0BDE8304000F088B848240220BD
:1012200080F937038C250220ED0F00088C2802205E
:1012300000440040B42402208C260220FD0F000848
:101240008C29022000480040202502208C27022003
:101250000D1000088C2A0220007800402E4B002937
:1012600008BF1946037C012B816630B50CD12B4B8E
:10127000984235D12A4B1A6C42F400321A641A6E25
:1012800042F400321A661B6E0A68036EC46D03EBEB
:101290005203B3FBF2F34A68150442BF23F007057B
:1012A00003F0070343EA4503E3608B6843F0400320
:1012B0006360CB68510543F00103A36042F4967369
:1012C00043F0010323604FF0FF33236205D512F092
:1012D00010221DD0B2F1805F1CD080F8643030BD88
:1012E000104B984208D10E4B1A6C42F480221A64BB
:1012F0001A6E42F48022C5E70B4B9842C4D1084BCA
:101300001A6C42F080421A641A6E42F08042B9E7C9
:101310007F23E2E73F23E0E7C43C000848240220A3
:1013200000380240B42402202025022000F160434E
:1013300000F01F020901400903F56143C9B28000B2
:1013400083F80013012300F16040934000F56140F1
:10135000C0F8803103607047F8B5154682680446CE
:101360000B46AA4200D28568A1692669761AB54261
:1013700007D218462A46FFF7EBFCA3692B44A3616A
:101380000DE011D9AF1B32461846FFF7E1FC3A4693
:10139000E1683044FFF7DCFCE2683A44A261A368EC
:1013A00028465B1BA360F8BD18462A46FFF7D0FC11
:1013B000E368E4E7836893422DE9F04104460F4671
:1013C000154600D2856860692669361AB54207D28B
:1013D0002A463946FFF7BCFC63692B4463610EE083
:1013E00013D9A5EB060832463946FFF7B1FC424651
:1013F000B919E068FFF7ACFCE26842446261A36897
:1014000028465B1BA360BDE8F0812A463946FFF7FA
:101410009FFCE368E2E7000010B50A440024C361C2
:10142000029B006040608460C16081614161026133
:10143000036210BD08B582694369934201D1826895
:1014400082B98268013282605A1C42611970426915
:1014500003699A4201D3C3684361002100F02EFF63
:10146000002008BD4FF0FF3008BD000070B52023FC
:1014700004460E4683F31188A568A5B1A368A26946
:10148000013BA360531CA36115782269934224BFDA
:10149000E368A361E3690BB120469847002383F317
:1014A0001188284670BD3146204600F0F7FE00281E
:1014B000E2DA85F3118870BD2DE9F74F05460F4636
:1014C00090469A46D0F81C90202686F311884FF05B
:1014D000000B144664B1224639462846FFF73CFF0C
:1014E000034668B95146284600F0D8FE0028F1D0DE
:1014F000002383F31188A8EB040003B0BDE8F08F4C
:10150000B9F1000F03D001902846C847019B8BF327
:101510001188E41A1F4486F31188DBE7C1608161FA
:1015200041611144C361009B0060406082600161C1
:1015300003627047F8B504460E461746202383F32E
:101540001188A568A5B1A368013BA36063695A1C13
:1015500062611E70236962699A4224BFE368636115
:10156000E3690BB120469847002080F31188F8BD4D
:101570003946204600F092FE0028E2DA85F3118811
:10158000F8BD0000836942699A4210B501D18268B2
:101590007AB98268013282605A1C82611C780369C0
:1015A0009A4201D3C3688361002100F087FE204680
:1015B00010BD4FF0FF3010BD2DE9F74F05460F4627
:1015C00090469A46D0F81C90202686F311884FF05A
:1015D000000B144664B1224639462846FFF7EAFE5E
:1015E000034668B95146284600F058FE0028F1D05D
:1015F000002383F31188A8EB040003B0BDE8F08F4B
:10160000B9F1000F03D001902846C847019B8BF326
:101610001188E41A1F4486F31188DBE702684368E7
:101620001143016003B11847704700001430FFF701
:1016300043BF00004FF0FF331430FFF73DBF000001
:101640003830FFF7B9BF00004FF0FF333830FFF7F5
:10165000B3BF00001430FFF709BF00004FF0FF31A7
:101660001430FFF703BF00003830FFF763BF0000FE
:101670004FF0FF323830FFF75DBF000000207047A9
:10168000FFF770BD044B0360002343608360C360B9
:1016900001230374704700BFDC3C000810B5202311
:1016A000044683F31188FFF7D9FD02232374002336
:1016B00083F3118810BD000038B5C36904460D4698
:1016C0001BB904210844FFF7A9FF294604F11400BF
:1016D000FFF7B0FE002806DA201D4FF48061BDE858
:1016E0003840FFF79BBF38BD026843681143016073
:1016F00003B118477047000013B5446BD4F8943415
:101700001A681178042915D1217C022912D119797E
:10171000012312898B4013420CD101A904F14C0022
:1017200001F03AFFD4F894440246019B21792068E5
:1017300000F0E0F902B010BD143001F0BDBE0000B1
:101740004FF0FF33143001F0B7BE00004C3001F011
:101750008FBF00004FF0FF334C3001F089BF000015
:10176000143001F08BBE00004FF0FF31143001F057
:1017700085BE00004C3001F05BBF00004FF0FF322F
:101780004C3001F055BF0000D0F8942438B51368F0
:1017900005461978042901D0012038BD017C0229B1
:1017A000FAD1127901205C8990400440F4D105F10E
:1017B000140001F01DFE02460028EDD0D5F8945427
:1017C0004FF480732868697900F082F9204638BDAB
:1017D000406BFFF7D9BF0000002070477047000042
:1017E0007FB5124B012502260446036000230574D1
:1017F00000F18402436029468360C3600C4B029071
:10180000143001934FF48073009601F0CDFD094B25
:1018100004F523722946019304F14C004FF48073C0
:101820000294009601F094FE04B070BD043D0008DF
:10183000D1170008F91600080B68202282F31188DE
:101840000A7903EB820210624A790D3243F82200D2
:101850008A7912B103EB820318620223C0F8941450
:101860000374002383F311887047000038B5037FA9
:10187000044613B190F85430ABB90125201D022164
:10188000FFF732FF04F1140025776FF0010100F03B
:1018900021FD84F8545004F14C006FF00101BDE8C3
:1018A000384000F017BD38BD10B5012104460430A2
:1018B000FFF71AFF0023237784F8543010BD00008F
:1018C00038B504460025143001F086FD04F14C00C3
:1018D000257701F055FE201D84F854500121FFF7B3
:1018E00003FF2046BDE83840FFF74EBF90F85C305C
:1018F00003F06003202B19D190F85D20212A0AD033
:10190000222A4FF000030ED0202A0FD1084A026588
:101910000722426504E0064B036507234365002365
:1019200083650120704703654365F9E70020704730
:1019300028220220D0F8943437B51A68044611786A
:1019400004291AD1017C022917D11979012312899E
:101950008B40134211D100F14C05284601F0D0FE16
:1019600058B101A9284601F017FED4F89444024664
:10197000019B2179206800F0BDF803B030BD000064
:1019800000EB8103F7B51C6A05460E46F4B120232F
:1019900083F3118805EB8607201D08214C34FFF7DF
:1019A000A3FEFB685B691B6813B1204601F002FED1
:1019B00001A9204601F0F0FD024648B1019B3146E5
:1019C000284600F097F8002383F3118803B0F0BD98
:1019D000FB685A691268002AF5D01B8A013B134044
:1019E000F1D105F15C02EAE70D3138B550F821403C
:1019F000DCB1202383F31188D4F89424136852793E
:101A000003EB8203DB689B695D6845B104216018C4
:101A1000FFF76AFE294604F1140001F0F3FC2046AA
:101A2000FFF7B2FE002383F3118838BD7047000032
:101A300001F0A2B8012300F1240200F13801037083
:101A40000023436042F8043B8A421361FAD10381C8
:101A50004381704738B50446202383F3118800255D
:101A60004160C560056145618561C561056201F040
:101A700093F80223237085F3118838BD70B500EB0D
:101A80008103054650690E461446DA6018B11022EB
:101A90000021FFF785F9A06918B110220021FFF796
:101AA0007FF931462846BDE8704001F03FB900009B
:101AB000028902F001020281428902F001024281A0
:101AC0000022026142618261C261026201F0C2B918
:101AD000F0B4012500EB810447898D40E4683D4363
:101AE000A469458123600023A2606360F0BC01F01B
:101AF000DDB90000F0B4012500EB810407898D40B9
:101B0000E4683D436469058123600023A26063604B
:101B1000F0BC01F057BA000070B50223002504465E
:101B20000370A0F8645080F8665080F86750058113
:101B30004581C560056145618561C561056280F8C3
:101B40004C5001F08FF863681B6823B1294620468A
:101B5000BDE87040184770BD0278436880F868207F
:101B600005221B6802700BB1042118477047000062
:101B7000436890F868201B6802700BB10521184774
:101B80007047000090F84C3070B5044613B1002344
:101B900080F84C3004F15C02204601F07DF9636866
:101BA0009B6863BB94F85C5015F0600615D194F8FF
:101BB0005D3005F07F0545EA032540F202339D4282
:101BC00000F00E815BD8022D00F0DC803FD8002DA4
:101BD00000F08780012D00F0CF800021204601F029
:101BE000C5FB0021204601F0B7FB63681B6813B1F9
:101BF000062120469847062384F84C3070BD2046C5
:101C000098470028CED094F8632094F8623043EAD5
:101C10000223626D934238BF636594F95C30656D51
:101C2000002B4FF0200380F2FD80002D00F0EC80AF
:101C3000092284F84C2083F311880021636D226D02
:101C40002046FFF757FF002383F3118870BDB5F5D9
:101C5000817F00F0B180B5F5407F49D0B5F5807F38
:101C6000BBD194F85E30012BB7D1B4F8643023F0C7
:101C70000203A4F8643026656665A665C3E740F2F2
:101C800001639D421ED8B5F5C06F3BD2B5F5A06F7C
:101C9000A3D1B4F85C30B3F5A06F0ED194F85E30E8
:101CA000204684F8663001F035F863681B6813B18C
:101CB0000121204698470323237000232365636591
:101CC000A365A0E7B5F5106F32D040F602439D4200
:101CD00052D0B5F5006F80D104F16703236501236D
:101CE00024E004F16403A5652365022363658AE7A4
:101CF00094F85E30012B7FF470AFB4F8643043F099
:101D00000203B6E794F861202046616894F86030D9
:101D10004D6843EA022394F85F1094F85E20A847C8
:101D200000283FF45AAF4368236503686365A4E75E
:101D30002378042B10D1202383F311882046FFF74A
:101D4000B7FE86F311886368032184F867601B6817
:101D500021700BB12046984794F85E30002BACD030
:101D600084F867300423237063681B68002BA4D0B9
:101D7000022120469847A0E7374B2365022363657D
:101D800000239DE794F86010204611F0800F01F0C9
:101D90000F010ED001F072F8012806D002287FF45E
:101DA0001CAF2E4B6065236567E72D4B656523658A
:101DB00063E701F055F8EFE794F85E30002B7FF40D
:101DC0000CAF94F8603013F00F013FF476AF1A06B1
:101DD000204602D501F0DEFA6FE701F0D1FA6CE798
:101DE00094F85E30002B7FF4F8AE94F8603013F076
:101DF0000F013FF462AF1B06204602D501F0B6FA90
:101E00005BE701F0A9FA58E7142284F84C2083F329
:101E100011882B462A4629462046FFF759FE85F3AE
:101E2000118870BD5DB1152284F84C2083F31188B0
:101E30000021636D226D2046FFF74AFE03E70B2267
:101E400084F84C2083F311882B462A4629462046E5
:101E5000FFF750FEE3E700BF343D00082C3D0008CB
:101E6000303D000838B590F84C300446152B29D881
:101E7000DFE803F03E28282828283E28280B2939A7
:101E800028282828282828283E3E90F8631090F813
:101E90006220436D42EA01229A4214D9C268128A32
:101EA000B3FBF2F502FB15356DB9202383F31188DE
:101EB0002B462A462946FFF71DFE85F311880A2383
:101EC00084F84C3038BD142384F84C30202383F33D
:101ED0001188002320461A461946FFF7F9FD002312
:101EE00083F3118838BD836D03B198470023E7E77A
:101EF000002101F03BFA0021204601F02DFA636831
:101F00001B6813B10621204698470623D8E7000036
:101F100090F84C20152A38B5044622D80123934066
:101F200040F6416213421DD113F480150FD19B027C
:101F300017D50B2380F84C30202383F311882B46D0
:101F40002A462946FFF7D6FD85F3118838BDC368B8
:101F50009B695B682BB9836D03B19847002384F8B4
:101F60004C3038BD002101F001FA0021204601F07B
:101F7000F3F963681B6813B10621204698470623CE
:101F8000EDE70000024B00221B605B609A60704727
:101F90008C2B0220002382680374054B1B68996810
:101FA0009142FBD25A6803604260106058607047EB
:101FB0008C2B022008B5202383F31188037C032B8C
:101FC00005D0042B0DD02BB983F3118808BD4369CC
:101FD00000221A604FF0FF334361FFF7DBFF00235D
:101FE000F2E790E80C001A6002685360F2E7000024
:101FF000002382680374054B1B6899689142FBD8E3
:102000005A68036042601060586070478C2B022051
:10201000054B196908741868026853601A601861E2
:1020200001230374FEF780B98C2B02204B1C30B5C2
:10203000054687B00A4C10D0236901A8094A00F070
:1020400065F92846FFF7E4FF049B13B101A800F0EF
:1020500099F92369586907B030BDFFF7D9FFF8E750
:102060008C2B0220B51F000838B50C4D0446416189
:102070002B6981689A68914203D8BDE83840FFF720
:1020800089BF1846FFF786FF01232C6101462374A0
:102090002046BDE83840FEF747B900BF8C2B022030
:1020A000044B1A681B6990689B68984294BF002093
:1020B000012070478C2B022010B5084C2368206942
:1020C0001A6854602260012223611A74FFF790FF9E
:1020D00001462069BDE81040FEF726B98C2B02208E
:1020E000FEE7000010B5194CFFF74CFF00F000F9B7
:1020F00080221749204600F085F8012344F8180C87
:102100000374144B144AD96821F4E0610904090CE2
:102110000A431249DA60CA6842F08072CA60104A03
:102120001049C2F8B01F116841F00101116010227E
:10213000DA77202283F82220002383F3118862B605
:102140000948BDE8104000F07FB800BFB42B022062
:10215000383D000800ED00E00003FA05F0ED00E076
:10216000001000E055CEACC5403D00082DE9F84F09
:102170001E4C4FF00008656904F11407C1464FF08A
:102180008043266AAA685B6A9E1B96421CD34FF066
:10219000200AAA68236AD5F80CB0B61A1344236241
:1021A0002B68BB425F606361C5F80C8001D101F010
:1021B000D1FA89F311882869D8478AF311886569AB
:1021C000AB689E42E5D2DAE76269BA420CD0916808
:1021D00023628E1B9660A86802282CBF1818981CD2
:1021E000BDE8F84F01F0BCBABDE8F88F8C2B022097
:1021F000034B59685A68521A9042FBD8704700BF87
:10220000001000E0826002220274002242747047D3
:102210008368A3F17C0243F80C2C026943F83C2C40
:10222000426943F8382C074A43F81C2CC268A3F1D2
:10223000180043F8102C022203F8082C002203F89F
:10224000072C70474103000810B5202383F3118841
:10225000FFF7DEFF00210446FFF706FF002383F3AC
:102260001188204610BD0000024B1B6958610F20E9
:10227000FFF7CEBE8C2B0220202383F31188FFF7BB
:10228000F3BF000008B50146202383F3118808201E
:10229000FFF7CCFE002383F3118808BD49B1064B3C
:1022A00042681B6918605A60136043600420FFF79E
:1022B000BDBE4FF0FF3070478C2B02200368984260
:1022C00006D01A680260506018465961FFF762BE76
:1022D0007047000038B504460D462068844200D19E
:1022E00038BD036823605C604561FFF753FEF4E787
:1022F000054B03F114025A619A614FF0FF32DA6123
:1023000000221A62704700BF8C2B0220F8B50361CF
:102310004FF08043C26002295C6A0646184B38BF02
:1023200002211A461F4652F8145F95420AD158619D
:1023300098611C620560456081600819BDE8F8403D
:1023400001F000BA186AAB68241A0C1902D3E41A17
:102350002D6804E09C4202D2204401F001FAAB68EF
:102360009C42F4D86B68356073601E604FF0FF3399
:102370006E60B460A968091BA960FB61F8BD00BF6D
:102380008C2B022010B41B4C234653F8141F81429F
:1023900010D0416802680A60026851609A424FF0AA
:1023A0000001C16003D0936881680B4493605DF8BD
:1023B000044B70470A6800209A4262615360C8600B
:1023C00003D15DF8044B01F0C5B9936888680344F4
:1023D000206A93604FF08042526A121A9342E6D903
:1023E000991A5DF8044B012998BF931C184401F019
:1023F000B7B900BF8C2B022000207047FEE7000019
:10240000704700004FF0FF3070470000022906D0EF
:10241000032906D00129064818BF00207047054847
:102420007047032A9ABF044800EBC200002070479F
:10243000303E0008E43D00083022022070B59AB01A
:1024400006460846144601AD294600F095F8284690
:10245000FEF79EFCC0B2431C5B0086E818002370A8
:102460000323023404F8013C00231946DAB2023493
:10247000904201D81AB070BDEA5C013304F8011C27
:1024800004F8022CF2E7000008B5202383F311883A
:102490000348FFF74FFA002383F3118808BD00BFFC
:1024A000482D022010B50446052916D8DFE801F0B2
:1024B00016150316161D202383F311880E4A0121D9
:1024C000FFF7DCFA20460D4A0221FFF7D7FA0C4845
:1024D000FFF7F6F9002383F3118810BD202383F35F
:1024E00011880748FFF7C2F9F4E7202383F3118826
:1024F0000348FFF7D9F9EDE7603D0008843D000887
:10250000482D022038B50C4D0C4C2A460C4904F1DC
:102510000800FFF793FF05F1CA0204F11000094912
:10252000FFF78CFF05F5CA7204F118000649BDE8F3
:102530003840FFF783BF00BF103202203022022054
:10254000B03D0008BD3D0008CB3D000870B5044615
:1025500008460D46FEF71CFCC6B22046013403783F
:102560000BB9184670BD32462946FEF7FBFB002822
:10257000F3D1012070BD00002DE9F04704460D465F
:10258000FEF706FC2B49C6B22046FFF7DFFF08B175
:102590000A36F6B228492046FFF7D8FF08B11036B0
:1025A000F6B2632E0BD8DFF88C80DFF88C90234FC7
:1025B000DFF894A0267846B92E70BDE8F087214652
:1025C0002846BDE8F04701F053BB252E2ED1072247
:1025D00041462046FEF7C6FB70B9194B2A4603F167
:1025E000100153F8040B8B4242F8040BF9D11B780D
:1025F000073411351370DDE7082249462046FEF7FF
:10260000B1FB98B9AA1C0F4B13F8011F023209093C
:102610005345C95D02F8041C197801F00F01C95D2A
:1026200002F8031CF0D118350834C3E72E700134CA
:102630000135BFE7503E0008CB3D00086A3E000868
:10264000583E00081FF4F01F2BF4F01FBFF34F8F0C
:10265000024AD368DB03FCD4704700BF003C024051
:1026600008B5074B1B7853B9FFF7F0FF054B1A6904
:10267000002A04DA044A5A6002F188325A6008BD1E
:102680006E340220003C02402301674508B5054B2B
:102690001B7833B9FFF7DAFF034A136943F00043AD
:1026A000136108BD6E340220003C02400B2870B557
:1026B00013D80B4A0B4C137863B94FF000610A4EE4
:1026C00044F8231056F8235001330C2B2944F7D13A
:1026D0000123137054F8200070BD002070BD00BFAE
:1026E000A0340220703402207C3E0008014B53F8D5
:1026F000200070477C3E00080C2070470B2810B566
:10270000044601D9002010BDFFF7D0FF064B53F857
:1027100024301844C21A0BB9012010BD12680132CE
:10272000F0D1043BF6E700BF7C3E00080B2810B553
:10273000044621D8FFF78AFFFFF792FF0F4AF323E1
:10274000D360C300DBB243F4007343F002031361B0
:10275000136943F480331361FFF778FFFFF7A6FF97
:10276000074B53F8241000F0DBF8FFF78FFF2046EB
:10277000BDE81040FFF7C2BF002010BD003C024082
:102780007C3E00082DE9F84312F0010315463FD1C5
:102790008218B2F1026F3BD22B4B1B6813F001037E
:1027A00036D0FFF75DFF294CF32340F20127E360A9
:1027B000FFF74CFF032D01D9830712D00F46401AB3
:1027C000224C40F20118EB1BC6190B44012B236964
:1027D00024D823F001032361FFF758FF0120BDE84F
:1027E000F883236923F44073236123693B43236106
:1027F00051F8046B0660BFF34F8FFFF727FF0368A4
:102800009E4208D0236923F001032361FFF73EFFB6
:102810000020BDE8F883043D0430CBE723F4407387
:10282000B9462361236943EA0803236137F8023B71
:102830003380BFF34F8FFFF709FF3688B6B2B9F880
:102840000030B342BFD0DDE700380240003C024018
:10285000084908B50B7828B153B9FFF701FF0123E8
:102860000B7008BD23B10870BDE80840FFF70EBF2C
:1028700008BD00BF6E34022002440439064BD2B2B8
:1028800010B5904200D110BD441C00B253F8200096
:1028900041F8040FE0B2F4E750280040104B30B587
:1028A0001C6F240407D41C6F44F400741C671C6F55
:1028B00044F400441C670B4C024404392368D2B230
:1028C00043F480732360084B904200D130BD441C18
:1028D00051F8045F00B243F82050E0B2F4E700BFC3
:1028E00000380240007000405028004007B5012227
:1028F00001A90020FFF7C0FF019803B05DF804FBB9
:1029000013B50446FFF7F2FFA04206D002A9012248
:10291000002041F8044DFFF7C1FF02B010BD0000D8
:102920000144BFF34F8F064B884204D3BFF34F8F50
:10293000BFF36F8F7047C3F85C022030F4E700BF2D
:1029400000ED00E0034B1B689B0042BF0122024BDD
:102950001A70704774380240A1340220014B187875
:10296000704700BFA1340220064A536823F00103D8
:102970005360EFF30983683383F30988002383F3FB
:102980001188704730EF00E010B5202383F31188E1
:10299000104B5B6813F4006318D0F1EE103AEFF3BC
:1029A00009844FF0807344F84C3C0B4BDB6844F8CF
:1029B000083CA4F1680383F30988FFF771FB18B1A1
:1029C000064B44F8503C10BD054BFAE783F31188E1
:1029D00010BD00BF00ED00E030EF00E05103000843
:1029E00054030008F0B5BFF34F8FBFF36F8F1D4B3B
:1029F0000021C3F85012BFF34F8FBFF36F8F5A6996
:102A000042F400325A61BFF34F8FBFF36F8FC3F8A8
:102A10008410BFF34F8FD3F8802043F6E076C2F3E3
:102A2000C904C2F34E32A507520102EA060E284637
:102A300021464EEA0007013900F14040C3F86072B8
:102A40004F1CF6D1203A12F1200FEED1BFF34F8F79
:102A50005A6942F480325A61BFF34F8FBFF36F8FD0
:102A6000F0BD00BF00ED00E0FEE70000084A094BA2
:102A700009498B4204D3094A0021934205D3704788
:102A800052F8040F43F8040BF3E743F8041BF4E790
:102A90005C400008343502203435022034350220F1
:102AA000036F002230B51146C46E9D684FF0FF30B1
:102AB00004EB421301329542C3F80019C3F8101910
:102AC000C3F80809C3F8001BC3F8101BC3F8080BB0
:102AD000EED24FF00113C4F81C3830BD890141F02B
:102AE0002001016103699B06FCD41220FFF780BB23
:102AF000204B03EB80022DE9F047D2F80CE0461C96
:102B0000DD6EDEF8142005EB0636D2F800C005EBCA
:102B10004018516861450BD30123D5F8342803FAD6
:102B200000F022EA0000C5F834081846BDE8F08736
:102B3000ACEB0103BEF81040A34228BF2346D8F8EF
:102B40001849A4B2B3EB840F10D894681F46A4F1BF
:102B5000040959F804AF042FC6F800A001D9043FB6
:102B6000F7E71C440B4494605360D2E70020BDE8B3
:102B7000F08700BFA434022010B5054C2046FEF7B4
:102B800059FF4FF0A043E366024B236710BD00BF1F
:102B9000A4340220D03E00080378012B70B505460E
:102BA00050D12A4BC46E98421BD1294B0E21432091
:102BB0005A6B42F080025A635A6D42F080025A65A5
:102BC0005A6D5A6942F080025A615A6922F08002B5
:102BD0005A615B69FEF7AAFB1E4BE3601E4BC4F80B
:102BE00000380023EE6EC4F8003EC02323604FF48B
:102BF0000413A3633369002BFCDA01230C20336137
:102C0000FFF7F6FA3369DB07FCD41220FFF7F0FA7E
:102C10003369002BFCDA00262846A660FFF740FF48
:102C20006B68C4F81068DB68C4F81468C4F81C68E2
:102C30004BB90A4BA3614FF0FF336361A36843F0C4
:102C40000103A36070BD064BF4E700BFA43402206B
:102C5000003802404014004003002002003C30C015
:102C6000083C30C0F8B5C46E054600214FF0006640
:102C70002046FFF733FF296F00234FF001128F68C2
:102C80004FF0FF30C4F83438C4F81C2804EB43126A
:102C900001339F42C2F80069C2F8006BC2F808090C
:102CA000C2F8080BF2D20B68EA6E6B6763621023FE
:102CB0001361166916F01006FBD11220FFF798FA7F
:102CC000D4F8003823F4FE63C4F80038A36943F451
:102CD000402343F01003A3610923C4F81038C4F85B
:102CE00014380A4BEB604FF0C043C4F8103B084B5C
:102CF000C4F8003BC4F81069C4F800396B6F03F1E5
:102D0000100243F480136A67A362F8BDAC3E00086A
:102D100040800010C26E90F86610D2F8003823F49C
:102D2000FE6343EA0113C2F8003870472DE9F04111
:102D30000EB20D4600EB8608D8F80C100F6807F0AD
:102D40000303022B50D0032B50D03D4A3D4F012BA3
:102D500018BF1746C46E4FEA451E002205F1100C3D
:102D600004EB0E03C3F8102B8A69002A40D04A8A6C
:102D700005F158033A435B01E2500123D4F81C28C3
:102D800003FA0CF31343C4F81C38A64400234A6921
:102D9000CEF8103905F13F03002A39D00A8A04EB36
:102DA0008303898B9208012988BF4A43416F5618D3
:102DB00041EA02422946466720465A60FFF78EFEE6
:102DC000D8F80C301B8A43EA85531F4305F14803AA
:102DD0005B01E7500123D4F81C2803FA05F51543DD
:102DE000C4F81C58BDE8F081174FB3E7174FB1E79F
:102DF00004EB4613D3F8002B22F40042C3F8002B57
:102E00000123D4F81C2803FA0CF322EA0303BAE7DF
:102E100004EB83030E4A04EB461629465A6020460B
:102E2000FFF75CFED6F80039012223F4004302FAD2
:102E300005F5C6F80039D4F81C3823EA0505CFE7B4
:102E400000800010008004100080081000800C102A
:102E500000040002026F12684267FFF721BE000003
:102E60005831C36E49015B5813F4004004D013F489
:102E7000001F14BF01200220704700004831C36EBC
:102E800049015B5813F4004004D013F4001F14BF31
:102E9000012002207047000000EB8101CB68196A15
:102EA0000B6813604B6853607047000000EB8103B0
:102EB00030B5DD68AA691368D36019B9402B84BFA7
:102EC000402313606B8A1468C26E1C4402EB4110ED
:102ED000013C09B2B4FBF3F46343033323F003036F
:102EE00043EAC44343F0C043C0F8103B2B6803F0EF
:102EF0000303012B0ED1D2F8083802EB411013F472
:102F0000807FD0F8003B14BF43F0805343F0005360
:102F1000C0F8003B02EB4112D2F8003B43F00443FF
:102F2000C2F8003B30BD00002DE9F041244D0446BD
:102F3000EE6E06EB4013D3F8087B3807C3F8087B26
:102F40000AD5D6F81438190706D505EB84032146AF
:102F50002846DB685B689847FA072FD5D6F81438FF
:102F6000DB072BD505EB8403D968CCB98B69488A7C
:102F70005E68B6FBF0F200FB12628AB91868DA6884
:102F800090420DD2121A83E81400202383F3118893
:102F90000B482146FFF78AFF84F31188BDE8F081D2
:102FA000012303FA04F26B8923EA02036B81CB68E5
:102FB00023B121460248BDE8F0411847BDE8F08141
:102FC000A434022000EB81034A0170B5DD68C36EB2
:102FD0006C692668E66056BB1A444FF40020C2F8BC
:102FE00010092A6802F00302012A0AB20ED1D3F8AE
:102FF000080803EB421410F4807FD4F8000914BFD2
:1030000040F0805040F00050C4F8000903EB421239
:10301000D2F8000940F00440C2F800090122D3F8B8
:10302000340802FA01F10143C3F8341870BD19B92C
:10303000402E84BF4020206020681A442E8A8419C4
:1030400040F00050013CB4FBF6F440EAC440C6E74F
:10305000F8B504461E48C56E05EB4413D3F808695D
:10306000F107C3F8086917D5D5F81038DA0713D572
:1030700000EB8403D9684B691F68DA68974218D25D
:10308000D21B00271A605F60202383F3118821463A
:10309000FFF798FF87F31188330617D50123D5F87A
:1030A0003428A340134211D02046BDE8F840FFF772
:1030B0001FBD012303FA04F2038923EA02030381FB
:1030C0008B68002BE8D021469847E5E7F8BD00BFA4
:1030D000A43402209F482DE9F84FC56E04466E695E
:1030E000AB691E4016F4805F6E6105D0FEF714FDDB
:1030F000BDE8F84FFFF748BC002E12DAD5F8003EC5
:103100009B0705D0D5F8003E23F00303C5F8003E29
:10311000D5F804388F4823F00103C5F80438FEF7CA
:1031200027FD370502D58B48FEF716FDB0040CD5F8
:10313000D5F8083813F0060FEB6823F470530CBF72
:1031400043F4105343F4A053EB60310704D5636894
:10315000DB680BB17F489847F2026FD4B3020CD5FD
:10316000D4F86C8000274FF00109DFF8E8A1236F45
:10317000F9B29B688B4280F09C80F70619D5E16E0E
:103180000A6AC2F30A1702F00F0302F4F012B2F552
:10319000802F00F0B580B2F5402F0AD104EB8303F5
:1031A00001F58051DB68186A00231A469F4240F0FF
:1031B0009C803303D5F818481DD5E70302D50020BD
:1031C000FFF7B2FEA50302D50120FFF7ADFE6003B5
:1031D00002D50220FFF7A8FE210302D50320FFF746
:1031E000A3FEE20202D50420FFF79EFEA30202D551
:1031F0000520FFF799FE77037FF57AAFE60702D542
:103200000020FFF725FFA50702D50120FFF720FFCB
:10321000600702D50220FFF71BFF210702D503201C
:10322000FFF716FFE20602D50420FFF711FFA30601
:103230007FF55EAF0520FFF70BFF59E7D4F86C80F0
:1032400000274FF00109DFF80CA1236F5FFA87FB1D
:103250009B685B4582D308EB4B13D3F8002902F43B
:103260004022B2F5802F22D1D3F80029002A1EDA9D
:10327000D3F8002942F09042C3F80029D3F800297E
:10328000002AFBDB5946E06EFFF728FC228909FA89
:103290000BF322EA0303238104EB8B03DB689B68B7
:1032A00013B15946504698475846FFF721FC01375D
:1032B000CBE708EB4112D2F8003B03F44023B3F50F
:1032C000802F10D1D2F8003B002B0CDA628909FA6A
:1032D00001F322EA0303638104EB8103DB68DB680B
:1032E0000BB150469847013741E79C0700D10A6867
:1032F000072B03F101039EBF0270120A013055E74C
:10330000023301F5805104EB830252689069026830
:10331000D0F808C04068A2EB000E00221046974289
:103320000AD104EB830463689B699A683A449A6003
:103330005A6817445F603CE712F0030F00D1086839
:10334000964502F1010282BF8CF80000000A0CF1E0
:10335000010CE4E7A4340220C36E03EB4111D1F861
:10336000003B43F40013C1F8003B7047C36E03EB0E
:103370004111D1F8003943F40013C1F80039704706
:10338000C36E03EB4111D1F8003B23F40013C1F8E5
:10339000003B7047C36E03EB4111D1F8003923F4B1
:1033A0000013C1F80039704730B50433039C017233
:1033B000002104FB0325C361049B00600363059B9C
:1033C0004060C16042610261856104624262816263
:1033D000C162436330BD00000022416AC2604161A6
:1033E00001616FF001018262C262FEF773BF0000EB
:1033F00003694269934203D1C2680AB10020704751
:10340000181D7047036919600021C2680132C2604B
:10341000C269134482699342036124BF436A036112
:10342000FEF74CBF38B504460D46E3683BB1626910
:103430000020131D1268A3621344E36238BD237A8F
:1034400033B929462046FEF729FF0028EDDA38BDBA
:103450006FF00100FBE70000C368C269013BC36075
:103460004369134482699342436124BF436A4361C1
:1034700000238362036B03B11847704770B52023A4
:10348000044683F31188866A3EB9FFF7CBFF0546F1
:1034900018B186F31188284670BDA36AE26A13F852
:1034A000015B9342A36202D32046FFF7D5FF0023BE
:1034B00083F31188EFE700002DE9F84F04460E462C
:1034C00090469946202787F311880025AA46D4F80C
:1034D00028B0BBF1000F09D149462046FFF7A2FFF3
:1034E00020B18BF311882846BDE8F88FA16AA8EBBC
:1034F000050BE36A5B1A9B4528BF9B46BBF1400F57
:103500001BD9334601F1400251F8040B914243F8B4
:10351000040BF9D1A36A403640354033A362A26A56
:10352000E36A9A4202D32046FFF796FF8AF3118896
:103530004545D8D287F31188C9E730465A46FDF78A
:1035400007FCA36A5E445D445B44A362E7E70000B6
:1035500010B5029C04330172C36103FB04210023F4
:1035600000608362C362039B40600363049BC4608A
:1035700042610261816104624262436310BD0000E6
:10358000026A6FF00101C260426A42610261002278
:103590008262C262FEF79EBE436902699A4203D10B
:1035A000C2680AB100207047184650F8043B0B600F
:1035B00070470000C3680021C2690133C3604369DA
:1035C000134482699342436124BF436A4361FEF717
:1035D00075BE000038B504460D46E3683BB123696B
:1035E00000201A1DA262E2691344E36238BD237A07
:1035F00033B929462046FEF751FE0028EDDA38BDE2
:103600006FF00100FBE7000003691960C268013A2E
:10361000C260C269134482699342036124BF436A52
:10362000036100238362036B03B1184770470000F6
:1036300070B5202304460E4683F31188856A35B998
:103640001146FFF7C7FF10B185F3118870BDA36A5B
:103650001E70A36AE26A01339342A36204D3E16954
:1036600020460439FFF7D0FF002080F3118870BD99
:103670002DE9F84F04460D4691469A464FF0200832
:1036800088F311880026B346A76A4FB951462046F1
:10369000FFF7A0FF20B187F311883046BDE8F88F0F
:1036A000A06AA9EB0603E76A3F1A9F4228BF1F469C
:1036B000402F1BD905F1400355F8042B9D4240F8DB
:1036C000042BF9D1A36A40364033A362A26AE36AAD
:1036D0009A4204D3E16920460439FFF795FF8BF342
:1036E00011884E45D9D288F31188CDE729463A464C
:1036F000FDF72EFBA36A3D443E443B44A362E5E74D
:10370000026943699A4203D1C3681BB918467047DE
:103710000023FBE7836A002BF8D0043B9B1AF5D00B
:103720001360C368013BC360C3691A4483699A424A
:10373000026124BF436A0361002383620123E5E73A
:1037400000F0AEB84FF08043002258631A610222A5
:10375000DA60704700224FF08043DA607047000063
:103760004FF08043586370474B6843608B688360B9
:10377000CB68C3600B6943614B6903628B69436229
:103780000B6803607047000008B5274B40F2FF71DB
:1037900026481A690A431A611A6922F4FF6222F064
:1037A00007021A611A691A6B0A431A631A6D0A43EF
:1037B0001A651F4A1B6D1146FFF7D6FF1D4802F11F
:1037C0001C01FFF7D1FF1C4802F13801FFF7CCFFC5
:1037D0001A4802F15401FFF7C7FF194802F17001BE
:1037E000FFF7C2FF174802F18C01FFF7BDFF164833
:1037F00002F1A801FFF7B8FF144802F1C401FFF776
:10380000B3FF134802F1E001FFF7AEFF114802F1E8
:10381000FC01FFF7A9FF104802F58C71FFF7A4FF28
:10382000BDE8084000F09EB80038024000000240A9
:10383000DC3E00080004024000080240000C024088
:10384000001002400014024000180240001C024018
:1038500000200240002402400028024008B500F089
:10386000F5F9FEF73FFCFFF76DF8BDE80840FEF7FD
:1038700049BE0000704700004FF080431A6992076C
:1038800010B508D500241C61202383F31188FEF7AE
:103890006DFC84F31188BDE81040FFF775B8000097
:1038A000104B08211C201A6C42F001021A641A6E97
:1038B00042F001021A660C4A1B6E936843F0010342
:1038C00093604FF080436B229A624FF0FF32DA62CE
:1038D00000229A615A63DA605A6001225A611A60C2
:1038E000FDF724BD00380240002004E01B4B4FF0E0
:1038F000FF3000211A696FEA42526FEA52521A6190
:103900001A69C2F30A021A611A695A6958615A6936
:1039100059615A691A6A62F080521A621A6A02F090
:1039200080521A621A6A5A6A58625A6A59625A6A04
:103930000B4A106840F480701060186F00F44070FB
:10394000B0F5007F03D04FF48030186719675368D3
:1039500023F40073536000F059B900BF00380240EF
:1039600000700040354B4FF44041354A1A64354AE7
:1039700011601A6842F001021A601A689207FCD5B9
:103980009A6822F003029A602C4B19469A6812F04A
:103990000C02FBD1186800F0F90018609A601A68F0
:1039A00042F480321A600B689B03FCD54B6F43F0E6
:1039B00001034B67214B5A6F9007FCD5224A5A608E
:1039C0001A6842F080721A601E4B1A465968490400
:1039D000FCD5196841F4803119605368D803FCD5CF
:1039E000136843F400331360164A53689903FCD5F7
:1039F000124B1A689201FCD5144A40F207319A60C2
:103A000040F20112C3F88C200022C3F89020104A23
:103A100011609A6842F002029A60084B9A6802F0BC
:103A20000C02082AFAD15A6C42F480425A645A6E47
:103A300042F480425A665B6E704700BF0038024015
:103A40000004001000700040186C40090094883891
:103A5000003C0240084A08B5536911680B4003F066
:103A60000103536123B1054A13680BB150689847AD
:103A7000BDE80840FEF788BF003C0140C823022093
:103A8000084A08B5536911680B4003F002035361FB
:103A900023B1054A93680BB1D0689847BDE8084048
:103AA000FEF772BF003C0140C8230220084A08B557
:103AB000536911680B4003F00403536123B1054AB5
:103AC00013690BB150699847BDE80840FEF75CBF29
:103AD000003C0140C8230220084A08B55369116818
:103AE0000B4003F00803536123B1054A93690BB1FE
:103AF000D0699847BDE80840FEF746BF003C01404A
:103B0000C8230220084A08B5536911680B4003F026
:103B10001003536123B1054A136A0BB1506A9847E9
:103B2000BDE80840FEF730BF003C0140C82302203A
:103B3000174B10B55C691A68144004F478725A6126
:103B4000A30604D5134A936A0BB1D06A984760065E
:103B500004D5104A136B0BB1506B9847210604D55E
:103B60000C4A936B0BB1D06B9847E20504D5094A18
:103B7000136C0BB1506C9847A30504D5054A936CA0
:103B80000BB1D06C9847BDE81040FEF7FDBE00BFFA
:103B9000003C0140C82302201A4B10B55C691A682A
:103BA000144004F47C425A61620504D5164A136D30
:103BB0000BB1506D9847230504D5134A936D0BB193
:103BC000D06D9847E00404D50F4A136E0BB1506EC8
:103BD0009847A10404D50C4A936E0BB1D06E984758
:103BE000620404D5084A136F0BB1506F9847230441
:103BF00004D5054A936F0BB1D06F9847BDE81040CC
:103C0000FEF7C2BE003C0140C8230220062108B5D1
:103C10000846FDF78BFB06210720FDF787FB0621F1
:103C20000820FDF783FB06210920FDF77FFB062115
:103C30000A20FDF77BFB06211720FDF777FB062105
:103C40002820BDE80840FDF771BB000008B5FFF76C
:103C50004DFEFDF7B7F9FDF713FDFDF7E9FEFDF7A2
:103C6000BDFDFFF707FEBDE80840FFF769BD000096
:103C7000034611F8012B03F8012B002AF9D17047F4
:103C80001210121312110000482D022048240220A5
:103C9000B42402202025022053544D3332463F3FA6
:103CA0003F3F3F3F0053544D333246375B347C3502
:103CB0005D780053544D333246375B367C375D7840
:103CC000000000000096000000000000000000005E
:103CD00000000000000000000000000000000000E4
:103CE0004916000835160008711600085D16000810
:103CF0006916000855160008411600082D16000820
:103D00007D16000800000000551700084117000844
:103D10007D1700086917000875170008611700086B
:103D20004D17000839170008D917000800000000D7
:103D300001000000000000006D61696E00000000DD
:103D4000583D0008D02B0220482D02200100000021
:103D5000E12000080000000069646C6500000000BC
:103D6000020000000000000081190008E9190008A5
:103D700040004000E0310220F0310220020000004B
:103D80000000000003000000000000002D1A0008E1
:103D900000000000100000000032022000000000BF
:103DA0000100000000000000A43402200101020014
:103DB0004865782F50726F6669434E4300437562C1
:103DC0006559656C6C6F772D424C002553455249FF
:103DD000414C2500A52400080D240008ED1800081A
:103DE0008924000843000000EC3D0008090243005C
:103DF000020100C032090400000102020100052492
:103E0000001001052401000104240202052406001B
:103E100001070582030800FF09040100020A0000EF
:103E20000007050102400000070581024000000074
:103E300012000000383E000812011001020000408C
:103E4000AE2D021000020102030100000403090468
:103E500025424F41524425004375626559656C6C9B
:103E60006F772D626473686F74003031323334358C
:103E7000363738394142434445460000008000004F
:103E800000800000008000000080000000000200B0
:103E90000000040000000400000004000000040012
:103EA0000000040000000400000004000000000006
:103EB000851B0008651E0008111F00084000400017
:103EC0001C3502201C350220010000002C35022088
:103ED0008000000040010000050000000000802A72
:103EE00000000000AAAAAAAA00000000FFFF00002C
:103EF0000000000000A00A00000100000000000017
:103F0000AAAAAAAA00000000FFFF0000000000000B
:103F1000000000001400005400000000AAAAAAAA91
:103F200014000054FFFF000000000000000000002B
:103F300080699A0100000000AAAA8AAA405555018A
:103F4000FFFF000000707007777000000081020022
:103F500000000000AAAAAAAA00410100FFFF000079
:103F600000000080080000000000000000000000C9
:103F7000AAAAAAAA00000000FFFF0000000000009B
:103F8000000000000000000000000000AAAAAAAA89
:103F900000000000FFFF0000000000000000000023
:103FA0000000000000000000AAAAAAAA0000000069
:103FB000FFFF000000000000000000000000000003
:103FC00000000000AAAAAAAA00000000FFFF00004B
:103FD00000000000000000000000000000000000E1
:103FE00000000000000000000000000000000000D1
:103FF00000000000000000000000000000000000C1
:1040000000000000000000000000000000000000B0
:10401000FF00000000000000983C00083F00000086
:1040200049040000A53C00083F00000051040000C6
:10403000B33C00083F0000000096000000000800AC
:10404000040000004C3E00080000000000000000DA
:104050000000000000000000000000000000000060
:00000001FF
